:020000021000EC
:10F800000C9446FC0C9463FC0C9463FC0C9463FC19
:10F810000C9463FC0C9463FC0C9463FC0C9463FCEC
:10F820000C9463FC0C9463FC0C9463FC0C9463FCDC
:10F830000C9463FC0C9463FC0C9463FC0C9463FCCC
:10F840000C9463FC0C9463FC0C9463FC0C9463FCBC
:10F850000C9463FC0C9463FC0C9463FC0C9463FCAC
:10F860000C9463FC0C9463FC0C9463FC0C9463FC9C
:10F870000C9463FC0C9463FC0C9463FC0C9463FC8C
:10F880000C9463FC0C9463FC0C9463FC11241FBE69
:10F89000CFEFD0E1DEBFCDBF11E0A0E0B1E0E6E206
:10F8A000FFEF01E00BBF02C007900D92A630B10739
:10F8B000D9F712E0A6E0B1E001C01D92A831B1076E
:10F8C000E1F70C94F5FC0C9400FC80911001813060
:10F8D00009F054C05F9941C08091080190910901DD
:10F8E000A0910A01B0910B010097A105B10599F50E
:10F8F00080910C0190910D01A0910E01B0910F012A
:10F900000196A11DB11D80930C0190930D01A09350
:10F910000E01B0930F01E0E9F1E03197F1F720918A
:10F92000000130910101409102015091030128171B
:10F9300039074A075B0778F4809164008B7F8093D6
:10F940006400809165008B7F80936500E0910601E3
:10F95000F091070109955F9BBFCF81E090E0A0E0A7
:10F96000B0E08093080190930901A0930A01B0933D
:10F970000B018CB1992787FD9095089580E090E068
:10F980000895982F80911001813019F45D9BFECF6E
:10F990009CB908950E9465FC803231F484E10E9494
:10F9A000C1FC80E10E94C1FC0895CF93C82F0E9442
:10F9B00065FC803249F484E10E94C1FC8C2F0E94D6
:10F9C000C1FC80E10E94C1FCCF910895282F90E0F6
:10F9D000981750F430911001313019F45F9BFECF2D
:10F9E0008CB19F5F9217C0F30895CFEFD0E1DEBFD7
:10F9F000CDBF809164008460809364008091650035
:10FA00008B7F8093650080EA9FE00197F1F780E7A4
:10FA100091E1A1E0B0E08093000190930101A093F7
:10FA20000201B093030110920C0110920D0110928B
:10FA30000E0110920F01109208011092090110920C
:10FA40000A0110920B01000080911001882319F423
:10FA500081E08093100180911001813059F480E1A0
:10FA600089B91092900082E08BB986E0809395006E
:10FA700088E18AB9809164008460809364008091F9
:10FA800065008460809365000E9465FC803309F402
:10FA90007AC08133E1F40E9465FCC82F8032A1F75F
:10FAA00084E10E94C1FC81E40E94C1FC86E50E94C1
:10FAB000C1FC82E50E94C1FC8C2F0E94C1FC89E43C
:10FAC0000E94C1FC83E50E94C1FC80E5C8C18F3F54
:10FAD000F9F40E9465FCC82F8936B1F687E50E94CB
:10FAE000C1FC8C2F0E94C1FC82E70E94C1FC8C2FBC
:10FAF0000E94C1FC8EE60E94C1FC87E60E94C1FC08
:10FB000086E50E94C1FC81E30E94C1FC8AE0AAC193
:10FB1000803439F40E9465FC8638A8F10E9465FCA7
:10FB200032C08134A1F40E9465FC803809F445C0DC
:10FB3000813811F481E09DC1823811F48FE099C1C0
:10FB4000893819F0883909F093C183E092C1823471
:10FB500011F484E103C0853421F485E00E94E6FCC1
:10FB600012C0803581F0813571F0823561F08335C6
:10FB700051F0853559F40E9465FC809311010E9473
:10FB800065FC809312010E94CAFC7ECF8635B9F4D1
:10FB90000E9465FC182F0E9465FC0E9465FCC82F1E
:10FBA0000E9465FC103309F063C1CC2311F48EE18F
:10FBB00060C1C13011F487E95CC182E05AC184366A
:10FBC00009F0CFC00E9465FC809314020E9465FC7E
:10FBD00080931302809117028E7F809317020E94F8
:10FBE00065FC853429F480911702816080931702A7
:10FBF000C0E0D0E08091130290911402C817D90799
:10FC000078F403E111E00E9465FCF80181938F0113
:10FC100021968091130290911402C817D90798F386
:10FC20000E9465FC803209F02FCF8091170280FF7F
:10FC300026C0C0E0D0E08091130290911402C81752
:10FC4000D90708F08CC0E3E1F1E0A0911101B09177
:10FC500012018191082E0E9487FF809111019091DD
:10FC600012010196909312018093110121968091C7
:10FC7000130290911402C817D90738F370C080910D
:10FC8000120187FF04C081E08093160202C0109227
:10FC90001602809116028BBF809111019091120182
:10FCA000880F991F90931201809311018091130284
:10FCB00080FF09C0809113029091140201969093E5
:10FCC000140280931302F894E199FECF1127E0917A
:10FCD0001101F0911201C3E1D1E0809113029091E2
:10FCE0001402103091F40091680001700130D9F3D2
:10FCF00003E000936800E89500916800017001300E
:10FD0000D9F301E100936800E895099019900091FA
:10FD1000680001700130D9F301E000936800E895B4
:10FD20001395103898F01127009168000170013088
:10FD3000D9F305E000936800E89500916800017030
:10FD40000130D9F301E100936800E89532960297FB
:10FD500009F0C7CF103011F00296E5CF112484E1ED
:10FD60007EC0843709F06AC00E9465FC809314024B
:10FD70000E9465FC80931302809111019091120101
:10FD80002091170297FF02C0226001C02D7F2093AF
:10FD900017020E9465FC20911702853421F421602E
:10FDA000209317020DC02E7F20931702809111011E
:10FDB00090911201880F991F909312018093110165
:10FDC0000E9465FC803209F05FCE84E10E94C1FC94
:10FDD000C0E0D0E08091130290911402C817D907B7
:10FDE00008F03FC08091170280FF08C0A091110168
:10FDF000B09112010E947FFF802D13C08695E09183
:10FE00001101F091120180FD02C084910AC0CF015E
:10FE1000AA27BB2780509040AF4FBF4FABBFFC011C
:10FE200087910E94C1FC809111019091120101966D
:10FE300090931201809311012196CCCF8537A9F4BC
:10FE40000E9465FC803209F01FCE84E10E94C1FC53
:10FE50008EE10E94C1FC87E90E94C1FC82E00E9401
:10FE6000C1FC80E10E94C1FC0FCE863709F00CCEA8
:10FE700080E00E94D5FC08CE1F93CF930E9465FCC2
:10FE8000C82F0E94C1FC0E9465FC182F0E94C1FC73
:10FE9000C13614F0C75503C0C0330CF0C05311363F
:10FEA00014F0175503C010330CF01053C295C07FE7
:10FEB000C10F8C2F992787FD9095CF911F910895A1
:10FEC000CF93282F992787FD9095807F907044E0ED
:10FED000959587954A95E1F78A3014F0895A01C0C3
:10FEE000805DC22FCF70CA3014F0C95A01C0C05D06
:10FEF0000E94C1FC8C2F0E94C1FCCF910895E19912
:10FF0000FECFBFBBAEBBE09A11960DB20895E1994A
:10FF1000FECFBFBBAEBB0DBA11960FB6F894E29AF6
:06FF2000E19A0FBE0895F6
:06FF2600701101008000D3
:040000031000F800F1
:00000001FF
